:10000000A00187130713003083168600870183122F
:100010000711071587120130E0006021E00160211F
:100020000D212330D80003171E308F000130031339
:10003000D900BD21831203130130DB000130DC0045
:100040002330DD006F21532023282528013083121F
:100050000313EA00073C031C362831286A08EA0A21
:100060002A286A08393E840080012E2808000230C0
:10007000E900073C031D031C522841286908E90ACE
:10008000392887126908B83EE40008216808403E14
:10009000E400082187166908393E84000008E4005E
:1000A00008213E2808000730A200A1014A210710BC
:1000B000E50165083F3C031CAA2861286508E50A9C
:1000C00059282620D12183120313C1001430DD21C9
:1000D0008312031341087F39C1000310F100083077
:1000E0000311E321C200F1000830EF21F1004108C3
:1000F0007102FF3A013EC10007304202FF3A013E61
:10010000C40003171E308F0013300313FA2183122B
:1001100003134108012283120313C3004408393E2C
:100120008400430880000730E6004208E700003CF6
:100130000318A6289E28E703670897286608393E13
:100140008400FF3080006608E6039B286508E8000D
:1001500037205E280730A200A1014A210712871527
:10016000E50165083F3C031C0229B9286508E50A3A
:10017000B1282620D12183120313C1001430DD21C0
:100180008312031341087F39C1000310F1000830C6
:100190000311E321C200F1000830EF21F100410812
:1001A0007102FF3A013EC10007304202FF3A013EB0
:1001B000C40003171E308F0013300313FA2183127B
:1001C00003134108012283120313C3004408393E7C
:1001D0008400430880000730E6004208E700003C46
:1001E0000318FE28F628E7036708EF286608393E5B
:1001F0008400FF3080006608E603F3286508E80005
:100200003720B62807146430DD2183120313080059
:1002100064088600871787130800E1016108013C24
:10022000031C49291629E10A61080E298712610871
:1002300003191D29071287151F29071687113F303B
:10024000E4000821B830E4000821C030E4000821AF
:10025000E3016308073C031C48293129E30A6308CA
:10026000292987124030E40008216308B83EE400E1
:1002700008218716E20162083F3C031C47294329F5
:10028000E20A62083B292008E400082140292E29BF
:100290001329080021083F3C03185129071287152C
:1002A00053290716871187122208B83EE400082157
:1002B0003F30A1052108403EE400082187160800D0
:1002C0006008031966290716871168290712871520
:1002D0003F30E4000821C030E400082108005B083A
:1002E000FF3EA1005C08FF3EA2004A2100005D081D
:1002F0008400DD0A0008DE00031D7F29BA290317E8
:100300001E308F001B300313FA21831203135E0883
:10031000E03EDE000122831203130310DE0D5E08AF
:100320000122831203135E08012283120313DF01EB
:100330005F08053C031CB929A029DF0A5F0898293A
:10034000071EA3294A215F08053C031DA929DE01D8
:10035000B2295F08003C013003180001012283121A
:100360000313DE0020085E06E40008212108A10A2C
:100370009D29762983120313080058088400590820
:1003800003178D0083168C170C14C62983120C08D2
:100390008000031908008D0A03198F0A8316840A46
:1003A000C42941309F0083160E309F0083121F1511
:1003B0000C1FD8290C131E080800F200DF29F20BCD
:1003C000DE29E2290800FF39031DE729FF34F30184
:1003D000F1020318ED2973080800F30AE829FF3930
:1003E000031DF3290034F300710800017107F30BBA
:1003F000F629080003178D0083168C13831203134C
:10040000080003178D0703188F0A83168C170C1426
:10041000831200000C0803130800FF3FFF3FFF3F5B
:103C020020005200580020005000610020006E0089
:103C12006F00720061006D0069007100750065003F
:103C2200200000008000C000E000F000F800FC006E
:103C3200FE00FF0000000000000000000000000085
:103C420000005F0000000000000007000000070005
:103C5200000014007F0014007F00140024002A00DA
:103C62007F002A0012002300130008006400620093
:103C720036004900550022005000000005000300F4
:103C82000000000000001C002200410000000000B3
:103C9200410022001C00000008002A001C002A002B
:103CA2000800080008003E0008000800000050005C
:103CB20030000000000008000800080008000800AA
:103CC200000030003000000000002000100008005A
:103CD200040002003E005100490045003E00000081
:103CE20042007F0040000000420061005100490094
:103CF20046002100410045004B003100180014002D
:103D020012007F00100027004500450045003900E1
:103D12003C004A00490049003000010071000900DE
:103D2200050003003600490049004900360006003C
:103D32004900490029001E0000003600360000003C
:103D420000000000560036000000000000000800DD
:103D52001400220041001400140014001400140086
:103D6200410022001400080000000200010051007E
:103D72000900060032004900790041003E007E0041
:103D82001100110011007E007F0049004900490026
:103D920036003E0041004100410022007F00410008
:103DA200410022001C007F004900490049004100F7
:103DB2007F0009000900010001003E0041004100AE
:103DC200510032007F000800080008007F00000058
:103DD20041007F00410000002000400041003F0000
:103DE20001007F0008001400220041007F00400013
:103DF2004000400040007F000200040002007F00FB
:103E02007F000400080010007F003E0041004100D6
:103E120041003E007F0009000900090006003E0043
:103E22004100510021005E007F00090019002900B5
:103E320046004600490049004900310001000100E6
:103E42007F00010001003F004000400040003F00B1
:103E52001F002000400020001F007F0020001800EB
:103E620020007F00630014000800140063000300B8
:103E7200040078000400030061005100490045007D
:103E82004300000000007F004100410002000400E6
:103E9200080010002000410041007F0000000000E7
:103EA2000400020001000200040040004000400043
:103EB2004000400000000100020004000000200059
:103EC20054005400540078007F004800440044002D
:103ED2003800380044004400440020003800440008
:103EE200440048007F003800540054005400180079
:103EF20008007E00090001000200080014005400BE
:103F020054003C007F000800040004007800000018
:103F120044007D00400000002000400044003D00BD
:103F2200000000007F001000280044000000410053
:103F32007F00400000007C000400180004007800AC
:103F42007C000800040004007800380044004400AB
:103F5200440038007C00140014001400080008001B
:103F62001400140018007C007C0008000400040007
:103F720008004800540054005400200004003F0090
:103F82004400400020003C004000400020007C0033
:103F92001C002000400020001C003C0040003000BB
:103FA20040003C00440028001000280044000C009F
:103FB2005000500050003C004400640054004C008B
:103FC200440000000800360041000000000000002C
:103FD2007F000000000000004100360008000000E1
:103FE200080008002A001C00080008001C002A0023
:0E3FF2000800080000000000000000000000B1
:08400000F73FF33FF03FF03FF2
:02400E00723D01
:00000001FF
